:100000000C9423070C945B070C945B070C945B0720
:100010000C945B070C945B070C945B070C945B07D8
:100020000C945B070C945B070C9476170C94B81631
:100030000C943D230C945B070C945B070C945B07BA
:100040000C945B070C945B070C945B070C945B07A8
:100050000C945B070C94F0220C945B070C945B07E8
:100060000C945B070C945B070C945B070C945B0788
:100070000C945B070C945B070C945B070C945B0778
:100080000C945B070C945B070C945B070C945B0768
:100090000C945B070C945B070C945B070C945B0758
:1000A0000C945B070C945B070C945B07B20A260B5D
:1000B000BA0A840A880ABE0A8B0AC10ACC0A960ABE
:1000C0001C0B9A0AD00A9E0AD40AFE0AA20AD80A6F
:1000D000080BA80ADE0AE80A8F0AC50A920AC80AAB
:1000E000AD0AE30AF40A140B160B800AB60A2F0BAA
:1000F0004F0B550B420A490B5B0B610B670B1A0C3C
:100100001A0C4C0C4C0CCB0CE70CE80DE80DEC0C6D
:10011000600D710D710D9A119D11D811E811EF113B
:10012000FA1198129812981298129812FD11FF1154
:1001300004122A124D12501253127712CA14F114DB
:10014000A016F114A0163D156015A01656166616D9
:10015000182902292C297E28EB29EB29FF28EB29D5
:10016000EB295A29EB296D29C429EB29EB29EB2925
:10017000EB299829EB29EB298929EB294729EB2938
:10018000EB29E529E529E529E529E529E529E529F9
:10019000E529E529E729EB291829F328EB29EB299B
:1001A000EB29EB29EB29EB29EB29EB29EB29EB29AF
:1001B000E729EB29EB29FF28EB29E329E329E329A8
:1001C000E329E329E329E329E329E329E7290000D7
:1001D000000000000000000000000000000000001F
:1001E000000000000000000000000000000000000F
:1001F00000007E0F00D4FFFFFFC700000078000062
:100200000000000000002A2B280000000000000071
:1002100000000000000000000029000000002C1E6B
:100220003420212224342627252E362D3738271E28
:100230001F202122232425263333362E37381F044E
:1002400005060708090A0B0C0D0E0F1011121314E6
:1002500015161718191A1B1C1D2F3130232D3504A4
:1002600005060708090A0B0C0D0E0F1011121314C6
:1002700015161718191A1B1C1D2F3130354C444503
:100280004255473A2064697361626C65642E0A00C6
:1002900044454255473A20656E61626C65642E0A9A
:1002A0000073757370656E64696E67206B65796243
:1002B0006F6172640D0A000A002530313662003A1F
:1002C000200025303258000A722F6320303132333B
:1002D0003435363738394142434445460A006C6567
:1002E000645F7461736B3A20253032580A0006311E
:1002F000FF0974A1010975150026FF0095207508F6
:100300008102C005010902A10185020901A10005C0
:1003100009190129081500250195087501810205B3
:1003200001093009311581257F950275088106097B
:10033000381581257F950175088106050C0A38025C
:100340001581257F950175088106C0C005010980CA
:10035000A101850319012AB700150126B7009501EF
:1003600075108100C0050C0901A101850419012A3D
:10037000A002150126A002950175108100C005019B
:100380000906A1018506050719E029E715002501E1
:100390009508750181020507190029EF150025014F
:1003A00095F075018102050819012905950575016A
:1003B0009102950175039101C00660FF0961A101D9
:1003C0000962150026FF0095207508810209631552
:1003D0000026FF00952075089102C005010906A1BD
:1003E00001050719E029E715002501950875018128
:1003F000029501750881010507190029FF150026DE
:10040000FF009506750881000508190129051500EA
:100410002501950575019102950175039101C05B58
:10042000435D005B445D005B535D005B575D005BBB
:10043000525D0009027400040100A0FA09040000E2
:1004400001030101000921110100012244000705F7
:1004500081030800010904010002030000000921D2
:100460001101000122220007058203200001070577
:100470000303200001090402000103000000092118
:100480001101000122B600070584032000010904C0
:1004900003000103000000092111010001221500E1
:1004A0000705850320000112010002000000084535
:1004B000415D06010001020001260343006F006E4A
:1004C000007300740065006C006C006100740069CA
:1004D000006F006E002000520065007600330000BF
:1004E0000012034100450042006F00610072006489
:1004F0000073000000040309043F00433E20004F46
:100500006E6573686F743A206163746976653A202A
:1005100025640A000A002530325820006E6B726F85
:100520005F7265706F72743A2025303258207C20DB
:10053000000A002530325820006B6579626F6172C5
:10054000645F7265706F72743A2025303258207C77
:1005500020004C25640A0029001E001F00200021F5
:10056000002200230024002500260027002D002E55
:100570000031004A002B0014001A00080015001773
:10058000001C0018000C00120013002F0030002A7D
:10059000004B00E00004001600070009000A000BF1
:1005A000000D000E000F003300340028004C004EF8
:1005B00000E1001D001B00060019000500110010DD
:1005C000003600370038000000E50052004D00E022
:1005D00000E300E200000000002C0000000000002A
:1005E00000E600E4000000500051004F0035003AE2
:1005F000003B003C003D003E003F00400041004207
:100600000043004400450049000100390001000199
:100610000001000100010001000100460047004800
:100620000001000100010001000100AA00A900A8CA
:1006300000B0000100010001000100010001000103
:100640000001004C00010001000100010001000157
:100650000001000100010001000100010000000193
:100660000001000100010001000100000000000184
:100670000000000000000001000100000001000176
:100680000001000100010001000100010001000162
:100690000001000100010001000100010001000152
:1006A0000001000100010001000100010001000142
:1006B0000001000100010001000100010001000132
:1006C0000001000100010001000100010001000122
:1006D0000001000100010001000100010001000112
:1006E0000001000100010001000100010001000102
:1006F00000010000000100010001000100010001F3
:1007000000000000000100000000000000010001E6
:1007100000000001000100010001000100010001D2
:1007200000010001000100010001000100010001C1
:1007300000010001000100010001000100010001B1
:1007400000010001000100010001000100010001A1
:100750000001000100010001000100010001000191
:100760000001000100010001000100010001000181
:100770000001000100010001000100010001000171
:100780000001000100010001000000010001000162
:100790000001000100010000000000010000000055
:1007A000000000010001000000010001000100291B
:1007B0000A002575002F002575005D2800256400BE
:1007C0002000256400200025640020002564007CB2
:1007D0000025303258006D6F7573656B6579205B4D
:1007E00062746E7C782079207620685D287265704E
:1007F0002F61636C293A205B006164645F6B6579EB
:100800005F6269743A2063616E2774206164643AA0
:1008100020253032580A0064656C5F6B65795F6231
:1008200069743A2063616E27742064656C3A2025F0
:100830003032580A006B65796D61705F636F6E6668
:1008400069672E7261773A20253032580A2E737705
:1008500061705F636F6E74726F6C5F636170736CF5
:100860006F636B3A2025750A2E636170736C6F633A
:100870006B5F746F5F636F6E74726F6C3A20257577
:100880000A2E737761705F6C63746C5F6C67756957
:100890003A2025750A2E737761705F7263746C5FFE
:1008A000726775693A2025750A2E737761705F6CDF
:1008B000616C745F6C6775693A2025750A2E7377D1
:1008C00061705F72616C745F726775693A2025753B
:1008D0000A2E6E6F5F6775693A2025750A2E737749
:1008E00061705F67726176655F6573633A20257535
:1008F0000A2E737761705F6261636B736C617368FA
:100900005F6261636B73706163653A2025750A2EBF
:100910006E6B726F3A2025750A2E737761705F6572
:1009200073636170655F636170736C6F636B3A20B2
:1009300025750A0064656275675F636F6E66696737
:100940002E7261773A20253032580A2E656E616228
:100950006C653A2025750A2E6D61747269783A20AB
:1009600025750A2E6B6579626F6172643A20257570
:100970000A2E6D6F7573653A2025750A00656563EB
:100980006F6E6669673A0A64656661756C745F6C60
:10099000617965723A2025750A000A092D204D619A
:1009A000676963202D0A443A094465627567204DE2
:1009B00065737361676520546F67676C650A583AA1
:1009C000094D6174726978204465627567204D6FC6
:1009D000646520546F67676C65202D2053686F77BE
:1009E000206B65797072657373657320696E206D15
:1009F000617472697820677269640A4B3A094B65C1
:100A000079626F61726420446562756720546F6714
:100A1000676C65202D2053686F77206B6579707245
:100A2000657373207265706F72740A4D3A0944657C
:100A3000627567204D6F75736520546F67676C65CD
:100A40000A563A0956657273696F6E0A533A09532A
:100A500074617475730A433A094163746976617409
:100A60006520436F6E736F6C65204D6F64650A4639
:100A7000312D4631303A0953776974636820746FB9
:100A8000204C6179657220302D3920284631302084
:100A90003D204C30290A302D393A09537769746367
:100AA0006820746F204C6179657220302D390A47B7
:100AB000524156453A0953776974636820746F2030
:100AC0004C6179657220302028616C7465726E61AA
:100AD0007465290A423A094A756D7020746F204284
:100AE0006F6F746C6F616465720A4553433A094ACB
:100AF000756D7020746F20426F6F746C6F616465E8
:100B0000722028616C7465726E617465290A453AB9
:100B1000095072696E7420454550524F4D205365FF
:100B20007474696E67730A4241434B5350414345A5
:100B30003A09436C65617220454550524F4D0A4E4B
:100B40003A094E4B524F20546F67676C650A000A92
:100B5000092D20436F6E736F6C65202D0A4553433A
:100B60002F713A09717569740A6D3A096D6F757361
:100B7000656B65790A002573000A092D205374619D
:100B8000747573202D0A686F73745F6B6579626F7B
:100B90006172645F6C65647328293A20253032588D
:100BA0000A6B6579626F6172645F70726F746F63F4
:100BB0006F6C3A20253032580A6B6579626F61722A
:100BC000645F69646C653A20253032580A6B657938
:100BD0006D61705F636F6E6669672E6E6B726F3AE0
:100BE00020253032580A74696D65725F72656164E0
:100BF000333228293A202530386C580A003F004EFD
:100C00004B524F3A206F66660A004E4B524F3A20C5
:100C10006F6E0A000A6D6F7573653A206F66660A1B
:100C2000000A6D6F7573653A206F6E0A000A6B6576
:100C300079626F6172643A206F66660A000A6B65BA
:100C400079626F6172643A206F6E0A000A6D617496
:100C50007269783A206F66660A000A6D617472697B
:100C6000783A206F6E0A000A64656275673A206FF1
:100C700066660A000A64656275673A206F6E0A004C
:100C80000A0A4A756D70696E6720746F20626F6F13
:100C9000746C6F616465722E2E2E2000433E20001E
:100CA000436C656172696E6720454550524F4D0A2D
:100CB00000313A0964656C6179282A31306D7329F5
:100CC0003A2025750A323A09696E74657276616C4C
:100CD000286D73293A2025750A333A096D61785FCA
:100CE00073706565643A2025750A343A0974696D34
:100CF000655F746F5F6D61783A2025750A353A0932
:100D0000776865656C5F6D61785F73706565643A7F
:100D10002025750A363A09776865656C5F74696DD8
:100D2000655F746F5F6D61783A2025750A00703ACF
:100D3000097072696E742076616C7565730A643A25
:100D4000097365742064656661756C74730A7570E7
:100D50003A092B310A646E3A092D310A6C743A094A
:100D60002B31300A72743A092D31300A4553432F22
:100D7000713A09717569740A0A7370656564203D7A
:100D80002064656C7461202A206D61785F737065E2
:100D90006564202A2028726570656174202F207494
:100DA000696D655F746F5F6D6178290A7768657238
:100DB000652064656C74613A20637572736F723D6F
:100DC00025642C20776865656C3D25640A5365654C
:100DD00020687474703A2F2F656E2E77696B697076
:100DE000656469612E6F72672F77696B692F4D6F2C
:100DF0007573655F6B6579730A004D3E20004D2564
:100E0000753A25733E20003F0A003D2025750A00F3
:100E10003F0A0064656661756C74730A0025750A83
:100E2000003F0A000A092D2056616C756573202D5C
:100E30000A00710A000A092D204D6F7573656B65F4
:100E400079202D0A000011241FBECFEFDAE0DEBFAB
:100E5000CDBF04B603FE18C08091C7039091C803AC
:100E6000A091C903B091CA038730904BA740B04B03
:100E700059F41092C7031092C8031092C90310923C
:100E8000CA03E0E0F8E3099512E0A0E0B1E0EEE784
:100E9000F7E502C005900D92AC3AB107D9F723E00F
:100EA000ACEAB2E001C01D92A73CB207E1F70E9494
:100EB0005C0E0C94BD2B0C940000FF93EF93E0911B
:100EC000AC02F091AD02309709F00995EF91FF91D6
:100ED0000895FC018591803011F0EFDFFBCF08957C
:100EE000FF27E0E230E247FF0CC0419597FF09C0C1
:100EF000EDE26095709580959095611D711D811D45
:100F0000911D27FF02C0219530E350E2AA27660F0A
:100F1000771F881F991FAA1FA41710F0A41B6395A1
:100F20005A95A9F7AA3008F0A95FA05DAF93F39591
:100F3000611571058105910541F7ED3211F4EF93CB
:100F4000F395F21718F43F93F395FBCF8F91B5DF2C
:100F5000FA95E1F70895E991F9918591803021F0B2
:100F6000853219F0AADFF9CF089520E0E894559171
:100F70005532C1F3503311F4689455915A3348F403
:100F8000505390F3220F022E220F220F200D250F17
:100F9000F4CF0EF4219589919991533619F3533773
:100FA00029F1533559F1BC0188279927E8945C361B
:100FB00021F48991999168945591543639F446EF0A
:100FC0007EF077FF0DC08FEF9FEF0AC055374AE0E4
:100FD00039F0583540E121F0523642E009F00895E9
:100FE000FF93EF937DDFEF91FF91B7CFFF93EF93E7
:100FF000FC0181918030B9F360DFFBCFFF93EF9369
:1010000068DFF1CFDF93CF93CDB7DEB72596A3DFAF
:10101000CF91DF910895A6E0B0E0E1E1F8E00C9413
:10102000742B49835A8349815A81992361F0222381
:1010300051F0CA010E949119182F682F89819A8155
:101040000E94AB1B04C0CA010E94771B182F698144
:101050007A81812F0E94D91F2696E3E00C94902B71
:10106000ABE1B0E0E6E3F8E00C94732B4E8B5F8BC2
:10107000688F798F8A8F9B8F192F911110924B0354
:10108000DE011F9687E0FD0111928A95E9F786E05F
:10109000FE01769601900D928A95E1F70A8D002364
:1010A00041F021E04F85588969897A89C8010E94F9
:1010B0000B080B8B1C8B87E0FE013F96DE01189618
:1010C00001900D928A95E1F7CE0108960E94F019E1
:1010D00081112CC087E0FE013896DE011196019047
:1010E0000D928A95E1F76C85662301F120910F033B
:1010F00030E0C9010196877099274091480350E07C
:101100008417950761F16D8397E0929FD001939FBB
:10111000B00D1124A05FBC4FFE01319601900D92DD
:101120009A95E1F780930F030E942E1917E08091A2
:10113000480390910F038917F9F0189FC0011124FB
:10114000805F9C4F0E94F0198823B1F08091480382
:1011500090E001968770992780934803E8CF0E941A
:10116000631C10920F0310924803E8E0F3E087E05D
:10117000DF011D928A95E9F76B96E4E00C948F2BC2
:101180008295982F937344E0949F900111248C7C56
:1011900086958695282B822F8575880F2A7A269525
:1011A000822B08950E94631C2FEF84E39CE0215062
:1011B00080409040E1F700C000009CE088E10FB65D
:1011C000F894A895809360000FBE90936000FFCFC5
:1011D000A8E0B0E0EEEEF8E00C94652BFC01848111
:1011E000882309F465C57F0121E040815181628136
:1011F000738195810E940B088C01F70185818823FA
:1012000009F438C1C80197578038910508F054C1D6
:10121000003108F03FC18FEF93E00E94E62A811170
:1012200039C130E8A32E32E0B32E002379F0A114A7
:10123000F4E0BF0609F42EC1C5010E94E62A81111F
:1012400001C001502FEFA21AB20AEFCFCE010196D2
:101250002C0188E0F20111928A95E9F72AE0322EFA
:1012600085010F5F1F4FC5010E94E62A89831A82FC
:10127000882309F40FC1813009F041C06501F2E013
:10128000CF0ED11CC8010E94E62A8A83882309F464
:1012900001C19FEF980F933060F423E0A20EB11CC0
:1012A000C6010E94E62A8B83882309F4F3C01C82BE
:1012B00029C0843031F54E0133E0830E911C02E0E9
:1012C00010E056018FEFA81AB80AC6010E94E62A5C
:1012D000F40181934F01882309F4DCC08C3741F479
:1012E000E2E0F0E0EC0FFD1FE00FF11F10820AC0FA
:1012F0000F5F1F4F65010730110519F7CBC058016B
:1013000001C056018201F8012081222309F4A8CFEF
:10131000213009F053C08181813081F46801F2E00D
:10132000CF0ED11CF8018281893319F460E570E099
:1013300002C060E070E00E940C1E15C0823049F4CB
:101340006801F2E0CF0ED11CF80182810E94FF1CDF
:101350000AC0833051F46801F2E0CF0ED11CF801CD
:1013600082810E94A51C860182C0843019F00F5F23
:101370001F4F7DC0F80122810E5F1F4F80E090E07B
:1013800030E0205331092A30310568F4389EA0013D
:10139000399E500D1124C901840F951F0F5F1F4FF7
:1013A000F8012081EDCF009709F461C0EFE9FFE07B
:1013B0003197F1F700C000000197F5CFE22FF0E080
:1013C000E250FE4F2490822F86958695869590E078
:1013D000FC01E251FE4F64902770712C022E02C076
:1013E000759467940A94E2F7F1E06F227724FC0188
:1013F000E252FE4F8490912C022E02C09594879465
:101400000A94E2F731E083229924FC01E253FE4F73
:10141000C490D12C02C0D594C7942A95E2F781E0FC
:10142000C822DD246114710419F081EE0E94FF1CB2
:101430008114910419F086EE0E94FF1C60E070E0B8
:10144000822D0E940C1E8114910419F086EE0E94D8
:10145000A51C6114710419F081EE0E94A51CC11431
:10146000D10429F060E070E08CE20E940C1E0F5F56
:101470001F4F49CFF801E851FC47E730F10508F06C
:101480003EC103C106E221EE41EE6AE17CE7C701FD
:101490000E94812480914903877009F409C4F701EF
:1014A0008581882309F404C48091BB0382FF00C4B2
:1014B00082E00E94121CFCC3F801E851FC47E730AF
:1014C000F10508F4E2C01092B203C8019057839767
:1014D00008F003C184E090E00E94EE2A9093BB03E1
:1014E0008093BA03F801E150F047E232F10520F4AD
:1014F000EA5AFF4F0C94582B8091BA038160ACC01C
:101500008091BB038860B4C08091BA038260A4C09C
:101510008091BA0320C08091BA0388609DC08091F9
:10152000BB031EC08091BB038260A2C08091BA033E
:10153000806192C08091BA0380628EC08091BA03AC
:1015400080648AC00E94631C8091BA03806884C052
:101550008091BA03886084607FC08091BB03826001
:10156000816086C08091BA038E7F76C08091BB0374
:10157000877F7EC08091BA038D7F6EC08091BA0351
:1015800020C08091BA03877F67C08091BB031EC0D3
:101590008091BB038D7F6CC08091BA038F7E5CC04D
:1015A0008091BA038F7D58C08091BA038F7B54C05D
:1015B0000E94631C8091BA038F774EC08091BA035A
:1015C000877F8B7F49C08091BB038D7F8E7F50C00A
:1015D0008091BA0382FB222720F991E0922790FBA9
:1015E00082F990FB83F938C08091BB03982F9095C6
:1015F00091708E7F892B90FB81F93AC08091BA035C
:1016000086FB222720F991E0922790FB86F924C0DF
:101610000E94631C8091BA0387FB222720F991E086
:10162000922790FB87F918C061E001C060E08EE06E
:1016300090E00E94042B1EC08091BA0384FB2227F5
:1016400020F991E0922790FB84F906C08091BA03BB
:10165000982F909590FB80F98093BA030BC08091EE
:10166000BB0383FB222720F991E0922790FB83F9AB
:101670008093BB036091BA037091BB0384E090E058
:101680000E94222B0E94631C05CFE858FF4F0C9448
:10169000582B07E225EE45EE6BE17CE7F8CE06E23B
:1016A00021EE40EE68E17CE7F2CE07E225EE44EE63
:1016B00069E17CE7ECCE06E221EE42EE6CE17CE7EC
:1016C000E6CE07E225EE46EE6DE17CE7E0CE08E2ED
:1016D00021E045EE6EE17CE7DACE0631FCE71F073C
:1016E00061F5809174038A7A91E009F490E0909317
:1016F000AE02811112C089E20E94A5230BC00631FF
:101700002CE7120761F48091AE02811189C289E24F
:101710000E9466230E949C21BDCE85E3EDCF073752
:10172000FCE71F0711F481E005C008372CE712071A
:1017300061F582E00E94051C08C007373CE71307EB
:1017400009F070C281E00E94541C43E062E081E035
:101750000E94E31B9FCE03309CE7190709F49EC249
:1017600008F467C20B358CE7180709F49FC20C35E3
:101770009CE7190709F075C28091BB0382FB88279B
:1017800080F991E089270E94291CF7018581008159
:101790001181882349F0C8010E949119D82E682F21
:1017A000C8010E94AB1B04C0C8010E94771BD82E41
:1017B000B8018D2D0E94D91F0E94E71F8C01A82E11
:1017C000F701B580968092949FE099228091490319
:1017D000877001F1BB20F1F0812F807F803469F0A8
:1017E00080E2800F8830B0F0812F807E803229F433
:1017F000F1E0F01778F4992069F08091BB0382FF43
:1018000009C082E00E94121C809149038770DD2488
:10181000D3948111D12CC12EC2948FE0C8228C2D7B
:1018200090E08C30910508F0D3C1FC01E158FF4FE6
:101830000C94582B812F807F1F70882311F01295F4
:10184000107FBB20B9F0112309F4B0C180E2800FF2
:10185000883010F0A11006C090917403192B1093DA
:10186000740305C090914B03192B10934B030E94F6
:101870009C219CC1802F0E94A51C112309F4A8C1A2
:10188000005E083080F1AA2071F1109590914B0311
:10189000192310934B032AC0812F807F1F70803241
:1018A00011F01295107FAA2029F021E0A21609F468
:1018B0004DC058C08091BB0382FD1BC0BB2069F0A6
:1018C000112339F030917403312B309374030E944B
:1018D0009C2180E00E94FF1C7BC180E00E94A51C2F
:1018E000112309F475C1812F0E9495210E949C212A
:1018F0006FC1BB2081F09920C9F131E0931268C11A
:1019000030914A03812F8323181709F461C1312BC9
:1019100030934A035DC191105BC1812F0E94941CDA
:1019200030914A03812F832329F0812F809538231A
:1019300030934A032091AF02812F822309F448C1DA
:10194000312F309523232093AF0242C1BB2029F0D1
:1019500085E0891508F43CC109C094E0991508F4A4
:1019600037C115C0BB2031F0911020C1812F0E94DA
:101970009B1C2EC1992059F0093309F026C1EFEFC5
:10198000F7EE23E0E150F0402040E1F71CC1812F49
:101990000E94941C1DC1812F86958695837019F035
:1019A000813059F015C1BB2019F0C801937002C0F5
:1019B00080E090E00E94122411C1BB2019F0C80100
:1019C000937002C080E090E00E94ED2307C16B2D70
:1019D000802F0E94FA2902C1812F8370A9F5B110CE
:1019E000FBC0402F429546954770440F440F802F0F
:1019F0008F7090E09C01042E01C0220F0A94EAF738
:101A000004FF08C08FE090E001C0880F4A95EAF714
:101A1000809501C080E0169516951370123069F01C
:101A200088F490917503113019F0822B892302C03C
:101A3000922B892B0E94601CCFC0822B9091750342
:101A40008927F8CF822BF6CFBB2019F0812F817028
:101A500001C08695882309F4BFC0402F4295469562
:101A60004770440F440F802F8F7090E09C01042E2C
:101A700001C0220F0A94EAF704FF08C08FE090E04B
:101A800001C0880F4A95EAF7809501C080E016955D
:101A900016951370123059F078F49091BA02113003
:101AA00019F0822B892309C0922B892B06C0822B27
:101AB0009091BA02892701C0822B0E94E01B8CC042
:101AC0001F70BB2039F0812F0E94541C802F0E9470
:101AD0009B1C82C0802F0E94941C812F0E94051C99
:101AE0007BC0802F32EFA31681F13A1538F090EFCA
:101AF000A91659F0E1EFAE1619F154C0F3EFAF1685
:101B000059F124EFA216C1F04DC0BB2081F034E0A2
:101B1000391508F45DC01F7181E090E0012E01C00D
:101B2000880F0A94EAF79091BA02892720C085E0CD
:101B3000891508F44DC0EFCF8091BB0382FD1AC018
:101B4000BB2029F0812F8F7120C0BB20D9F3812FBA
:101B50008F710E94051C3CC0BB2041F01F7181E0C9
:101B6000012E01C0880F0A94EAF701C080E00E94AC
:101B7000E01B2EC0BB2061F0812F8F7198E0899F00
:101B8000900111242360209349030E94541C20C01B
:101B900081E00E94121CE1E0E915D0F482E00E948D
:101BA000121C16C0BB2021F0992061F2802F92CE2A
:101BB000992069F2893349F4FFEF27EE33E0F150C1
:101BC00020403040E1F700C00000802F0E94A51C9B
:101BD00088EF8C0D843010F40E943724DD20A9F0AA
:101BE0008091490380FD11C0F70115828695869585
:101BF00086950E94541CC7010E94E8088091490301
:101C00008695869586950E94051C20E0F701408107
:101C1000518162817381848195810E940B0848C043
:101C200085E376CD08378CE7180709F094CD82E07C
:101C30008ACD0130FCE71F07B9F1C8F401153CE774
:101C4000130709F0A2CD0E94631CFFEF24E33CE0E0
:101C5000F15020403040E1F700C000000E94CC224B
:101C600019CC0A351C4709F090CD81E08CCD8091CC
:101C7000B903982F9095917090FB80F98093B903E8
:101C8000992319F080E992E002C08EE792E09F93D9
:101C90008F930E9402080F900F90FCCB6FEF7FEFA5
:101CA00080E090E00E94222B0E94D20880E06BCD61
:101CB0002896E2E10C94812BA6E2B0E0E2E6FEE099
:101CC0000C94652B85B7806885BF85B7806885BF14
:101CD00084B7877F84BF0FB6F894A8958091600081
:101CE000886180936000109260000FBE90E080E8F1
:101CF0000FB6F89480936100909361000FBE87E760
:101D000093E19093AD028093AC020E94FC160E9476
:101D10001B178091E20084608093E20078948091A8
:101D2000E0028823A1F01091E9001F709091EC006F
:101D3000892F817090FD80E8182B1092E900809126
:101D4000E80083FD0E94E8131F701093E90082E011
:101D500084BD93E095BD9AEF97BD80936E000E947D
:101D60006824811102C00E94BB2601E111E046E116
:101D7000E42E41E0F42ED8018D918D018F3F11F0BA
:101D80000E940F1FE016F106B1F706E111E035E2FF
:101D9000E32E31E0F32EF80181918F018F3F11F096
:101DA0000E940F1FE016F106B1F78AE0E6ECF2E0C0
:101DB000DF01282F1D922A95E9F7E0EBF2E0DF0121
:101DC0001D928A95E9F780E090E00E94EE2A853E18
:101DD0009E4F21F40E946824811102C00E94282194
:101DE00082E090E00E94E62A8093B90384E090E0CC
:101DF0000E94EE2A9093BB038093BA030E94261F91
:101E0000EFEFF6E721E0E150F0402040E1F700C0BD
:101E100000000E94261F8091C60280FF08C06FEF5D
:101E20007FEF80E090E00E94222B0E94CC2283E092
:101E300090E00E94E62A0E94601C80E091E090936E
:101E4000B6038093B5038091E002853009F053C05A
:101E50008091B90380FF08C081EA92E09F938F933D
:101E60000E9402080F900F9000E112E18091E002C1
:101E7000853009F03CC08091E002843021F110925D
:101E8000BC0348E150E080E40FB6F894A895409375
:101E900060000FBE8093600083B7817F846083BF42
:101EA00083B7816083BF7894889583B78E7F83BF23
:101EB0000FB6F894A89580916000886180936000C7
:101EC000109260000FBE8091DF02882309F4CECF0C
:101ED0000E94261FE6ECF2E081919191892B09F096
:101EE00030C3A0EDB2E0AE17BF07B1F7BFCF0E947D
:101EF000631C0E9437240E94261F9BEBE92E92E070
:101F0000F92E26EC422E22E0522E25EC32E0D201B0
:101F1000F701419151918D919D91842795272E171D
:101F20003F0719F0892BA9F305C0892B19F40E94EA
:101F3000042193C08091B90381FD04C0912C7724C2
:101F400073944FC087EC92E09F938F930E94020896
:101F50000F900F90F6ECCF2EF2E0DF2E00E010E0B5
:101F6000AFEB8A2EA2E09A2EB9EBAB2EB2E0BB2EDD
:101F700087EB682E82E0782E1F930F93E2ECF2E05D
:101F8000FF93EF930E9402089F928F920E94020893
:101F9000D6018C9111962C90B2E0CB0ED11C0E94F0
:101FA000C008382E822D0E94C008232D30E0322F29
:101FB0002227F901E82BCF019F938F93BF92AF9215
:101FC0000E9402087F926F920E9402080F5F1F4FCB
:101FD0000FB6F894DEBF0FBECDBF0530110561F618
:101FE000ADCFD201AD90BD902D01F701C080D18061
:101FF000CA24DB24C114D10439F1812C01E010E0A2
:10200000C8018C219D21892BB1F089A29AA20E943E
:1020100031239CA38BA37DA291E098012A213B212F
:10202000232B09F490E09EA349A15AA16BA17CA1A6
:102030008DA10E9430088394000F111FFFE08F12C2
:10204000DFCFD701AD92BC929394B2E0EB0EF11CBE
:10205000E5E09E12C6CF0E94252386E0EAEAF3E07F
:102060008E010F5F1F4FD80101900D928A95E1F705
:10207000B090AB03C090AC03E090AD03D090AE0342
:10208000F090AF031092AC031092AD031092AE0328
:102090001092AF03C11003C0EE2009F454C0809128
:1020A000A8039091A9030E941623AC019091A50367
:1020B000992339F020910F0130E02417350758F0AB
:1020C00042C020911001FAE02F9F900111242417A3
:1020D000350718F038C09F3F19F09F5F9093A50314
:1020E000CC2061F00E9402261C1414F491E001C07F
:1020F0009FEF899F802D11248093AC03EE2061F027
:102100000E9402261E1414F09FEF01C091E0899FE7
:10211000802D11248093AD038091AC03882399F026
:10212000A090AD03AA2079F00E944126811101C040
:1021300081E08093AC038A2D0E944126811101C069
:1021400081E08093AD03D11003C0FF2009F447C0A4
:102150008091A6039091A7030E9416239C01909161
:10216000A303992309F40CC221353105C0F19F3F27
:1021700019F09F5F9093A303DD2061F00E94C925B1
:102180001D1414F491E001C09FEF899F802D11244C
:102190008093AE03FF2061F00E94C9251F1414F044
:1021A0009FEF01C091E0899F802D11248093AF03A0
:1021B0008091AE03882399F0A090AF03AA2079F014
:1021C0000E944126811101C081E08093AE038A2DD7
:1021D0000E944126811101C081E08093AF0380916C
:1021E000AB03B8121AC08091AC03882311F08C1194
:1021F00014C08091AD03882311F08E110EC0809120
:10220000AF03882311F0F81208C09091AE03992310
:1022100031F081E09D1104C002C081E001C080E086
:1022200080FD15C08091AC0381110FC08091AD037A
:1022300081110BC08091AE03811107C081E09091A4
:10224000AF03911103C080E001C081E080FD0E94D6
:102250000525BA82CB82EC82DD82FE8286E0F8011F
:10226000AAEAB3E001900D928A95E1F70E94372423
:10227000F82E8091C502F816B1F0F092C5020E94C6
:1022800025238091B90382FF0EC080FF0CC01F92EE
:10229000FF928EED92E09F938F930E9402080F9021
:1022A0000F900F900F908091E002843009F0CBCD19
:1022B00083E08093E9008091E80082FFC4CD8091A3
:1022C000E80085FF21C00E94B51881111BC060E2A3
:1022D000E62EF12C680109C08091F100D6018D93A2
:1022E0006D01B1E0EB1AF10869F08091E80085FD1D
:1022F000F3CF8091E8008B778093E8000E94B518B7
:10230000882399F391E001C090E08091E8008B77F9
:102310008093E800992309F496CDE9818E2F90E00F
:10232000FC013197E331F10508F002C1E557FF4F99
:102330000C94582B1A828CE065C08A81823009F493
:1023400016C150F4813009F0F3C00E9425239B830D
:102350008C837D836E83EEC0833041F0843009F03E
:10236000E7C01B821C821D821E82E4C04B81D80103
:1023700080E090E0242F30E0B901680F791F6530CC
:10238000710508F0D7C0E42FE80FF0E0EE0FFF1F53
:10239000EA53FD4F5081618113966C931397149605
:1023A0005C931497019612968E30910529F7C2C05E
:1023B0008A81823021F0853009F4BCC0B9C06B81BC
:1023C0007C818D819E810E945E2B0E944424B2C03C
:1023D0004C816B818A810E94CB269D83CFC02D8149
:1023E0003E813227232732274C816B818A810E94CC
:1023F0005F26A0C00E9486269DC080E152C081E079
:102400008A8380E88B8396C0EA80FB80FE24EF24D9
:10241000FE24AC80B12C6801C70180589D4F960105
:10242000201B310B2A153B0508F084C0E0E8EE16AE
:10243000E1E0FE0630F40E94E62AD60114968C9361
:1024400002C0F6011482FFEFEF1AFF0A2FEFC21A43
:10245000D20AE2CFEA80FB80FE24EF24FE24AC8087
:10246000B12C6801C70180589D4F9601201B310B8C
:102470002A153B0508F05EC040E8E41641E0F4068A
:1024800028F4D60114966C910E94042BBFEFEB1A2E
:10249000FB0AEFEFCE1ADE0AE5CF0E944F264AC0B4
:1024A00084E08A8347C0EA80FB80FE24EF24FE2478
:1024B000AC80B12C6801C70188969601201B310BB6
:1024C0002A153B05B8F5F8E5EF16F2E0FF0630F403
:1024D0000E94E62AD60114968C9302C0F60114825B
:1024E000FFEFEF1AFF0A2FEFC21AD20AE4CFEA80F9
:1024F000FB80FE24EF24FE24AC80B12C6801C701D0
:1025000088969601201B310B2A153B0598F448E567
:10251000E41642E0F40628F4D60114966C910E9469
:10252000042BBFEFEB1AFB0AEFEFCE1ADE0AE7CF60
:102530008FEF898340E250E0B80182E00E9473226D
:1025400082CC09BD19BD09B400FEFDCF8091D80031
:102550008F7D8093D8008091E00082608093E000BE
:102560008091E00081FDFCCF0E94631C7FCC87E25C
:1025700090E00E94E62A1B821C821D828E83DACFA5
:102580002B30310508F0F5CD2ACE8091E20287FF8D
:1025900011C08091E80082FD05C08091E0028111A8
:1025A000F8CF11C08091E8008B770BC08091E002DA
:1025B000882349F08091E80080FFF8CF8091E800FF
:1025C0008E778093E8000895982F973068F5909360
:1025D000E900981739F07091EC002091ED005091CE
:1025E000F00003C0242F762F50E021FD02C09F5F32
:1025F000ECCF3091EB003E7F3093EB003091ED005B
:102600003D7F3093ED003091EB0031603093EB0073
:102610007093EC002093ED005093F0002091EE00B9
:1026200027FDE5CF80E008958F708093E90081E079
:1026300008952091E8023091E9022617370748F003
:102640006115710539F42091E8002E772093E80098
:1026500001C0B901FC0120E06115710579F180919B
:10266000E0028823F1F18530F1F18091E80083FDEB
:102670003CC08091E80082FD2EC08091E80080FF80
:10268000EBCF2091F3008091F20090E0922B611546
:10269000710551F08830910538F421912093F100B3
:1026A000615071090196F3CF21E0089709F020E00D
:1026B0008091E8008E778093E800CECF2111CFCFB4
:1026C0000AC08091E002882361F0853061F080913A
:1026D000E80083FD0AC08091E80082FFF2CF80E02D
:1026E000089582E0089583E0089581E008959FB7FA
:1026F000F8941092D1029FBF9091E002943009F0BB
:1027000057C09091E9009F703091EC00232F217009
:1027100030FD20E8922B25E02093E9002091EB008A
:1027200020FF43C02091EE0027FF3FC02091D00240
:10273000222321F02091E80025FF37C01092D0021B
:1027400026E03091E80035FD15C03091E0023430CC
:1027500061F53091EB0035FD28C0215021F481E076
:102760008093D00222C0EFE9FFE03197F1F700C07B
:102770000000E7CF8093F1008091E80085FD0AC05A
:102780008091E80080FFFCCF8091E8008E778093F5
:10279000E80006C08FB7F89421E02093D1028FBFE4
:1027A0009F709093E90080E008959F709093E900F6
:1027B0008FEF089543E050E0BC0184E00E94732253
:1027C000089546E050E0BC0184E00E947322089521
:1027D000AAE2B0E0EEEEF3E10C94742BE2EEF2E04C
:1027E0008091F100819342E0EA3EF407C9F78091BD
:1027F000E302833009F463C030F4813071F0823039
:1028000009F49DC0B4C08A3009F489C08B3009F442
:102810006EC0893009F0ABC020C08091E202813ADD
:1028200009F0A5C08091E800877F8093E80080913F
:10283000E6029091E702892B21F468E086ED92E0B0
:1028400003C060E080E090E070E00E941913809186
:10285000E8008B778093E8008AC08091E2028132A1
:1028600009F085C08091E6029091E702009719F087
:10287000029709F07CC08091E800877F8093E80090
:102880008091E80082FD05C08091E0028111F8CFBF
:102890006EC02091F3008091F20090E0922B02979D
:1028A00031F48091F100813011F0863021F4809173
:1028B000F1008093D5028091E8008B7754C080911D
:1028C000E202813A09F053C08091E6029091E7025A
:1028D000892B09F04CC08091E800877F8093E80045
:1028E0008091E80080FFFCCF80910A0137C0809181
:1028F000E2028132E1F58091E6029091E702892BB4
:10290000B1F58091E800877F8093E8000E94C512AE
:102910008091E40280930A010E94631C28C0809188
:10292000E202813221F58091E800877F8093E80000
:102930000E94C5128091E5028093D40218C0809154
:10294000E202813AA1F48091E800877F8093E80059
:102950008091E80080FFFCCF8091D4028093F10049
:102960008091E8008E778093E8000E94C5128091E4
:10297000E80083FFE5C18091E2029091E302492FD4
:1029800050E04A30510508F0DBC1FA01E256FF4F32
:102990000C94582B803821F0823809F0D1C108C03E
:1029A0008091DE029091DF02992389F082600FC04E
:1029B0008091E6028F70873008F0C2C18093E900F1
:1029C0008091EB0085FB882780F91092E9009091B7
:1029D000E800977F9093E8008093F1001092F10057
:1029E00071C1282F2D7F09F0ABC1882319F08230E7
:1029F00061F0A6C18091E402813009F0A1C1933059
:102A000009F080E08093DF022EC08091E402811102
:102A10002AC08091E6028F702FEF280F263008F031
:102A20008FC18093E9002091EB0020FF1CC0933000
:102A300021F48091EB00806214C09091EB009061D2
:102A40009093EB0021E030E0A90102C0440F551F34
:102A50008A95E2F74093EA001092EA008091EB0039
:102A600088608093EB001092E9008091E800877FF6
:102A70008093E8000E94C51263C1811161C1109169
:102A8000E4021F778091E3008078812B8093E3003C
:102A90008091E800877F8093E8000E94C5128091B2
:102AA000E80080FFFCCF8091E30080688093E30022
:102AB000111102C082E001C083E08093E00240C1B6
:102AC0008058823008F03CC12091E4023091E50248
:102AD0002C3D53E0350779F583E08A838AE28983C8
:102AE0004FB7F894DE01139620E03EE051E2E32F69
:102AF000F0E050935700E49120FF03C0E295EF709F
:102B00003F5FEF708E2F90E0EA3010F0C79601C063
:102B1000C0968D939D932F5F243149F74FBF8091CD
:102B2000E800877F8093E8006AE270E0CE010196BA
:102B30000E941913B5C08091E6029091E702432FDD
:102B4000552743305105A9F068F44130510509F487
:102B500006C14230510509F0F3C084E790E0E3E399
:102B6000F4E04BC04132510529F14232510589F15F
:102B7000E7C0C901992781309105A1F058F002976B
:102B800009F0DEC0E9EBF4E0E4918E2F90E0E9EB90
:102B9000F4E030C0E5EFF4E0E4918E2F90E0E5EF53
:102BA000F4E028C0E1EEF4E0E4918E2F90E0E1EE55
:102BB000F4E020C08430910508F0C2C0880F991F4E
:102BC000FC01EF5CFE4F0190F081E02D89E090E088
:102BD00014C08430910508F0B3C0FC01EE0FFF1F54
:102BE000E75DFE4F0190F081E02DDC01AB5DBE4F53
:102BF0008C9190E0009709F4A3C02091E800277F12
:102C00002093E8002091E8023091E90282179307AF
:102C100008F49C0140E02115310589F18091E00222
:102C2000882309F43DC08530D9F18091E80083FD07
:102C300037C08091E80082FD2FC08091E80080FFBE
:102C4000EACF4091F3008091F20090E0942B21159F
:102C5000310559F08830910540F444914093F100DA
:102C60003196215031090196F2CF41E0089709F0E1
:102C700040E08091E8008E778093E800CCCF41114E
:102C8000CDCF0AC08091E002882351F0853041F019
:102C90008091E80083FD04C08091E80082FFF2CFBC
:102CA0008091E8008B778093E8004AC0803809F073
:102CB00047C08091E800877F8093E8008091E1021F
:102CC0008093F1008091E8008E77D2CE811138C0D8
:102CD0008091E4029091E502992702978CF580910A
:102CE000E800877F8093E8001091E4021093E102EE
:102CF0000E94C512111106C08091E30087FD02C039
:102D000081E001C084E08093E00242E061EC81E078
:102D10000E94E41242E261EC84E00E94E41242E28A
:102D200061EC82E00E94E41242E260EC83E00E94E7
:102D3000E41242E261EC85E00E94E4128091E0023C
:102D40008091E80083FF10C08091E800877F809326
:102D5000E8008091EB0080628093EB0005C082E187
:102D600090E0E7EAF4E049CFAA96E3E00C94902BD8
:102D70001F920F920FB60F9211242F933F934F93F0
:102D80005F936F937F938F939F93AF93BF93CF93F3
:102D9000DF93EF93FF93C091E900CF708091EC0037
:102DA000D82FD17080FDD0E81092E9008091F0001A
:102DB000877F8093F00078940E94E8131092E900D6
:102DC0008091F00088608093F000CD2BCF70C0938D
:102DD000E900FF91EF91DF91CF91BF91AF919F916A
:102DE0008F917F916F915F914F913F912F910F90B4
:102DF0000FBE0F901F901895E8EDF0E080818E7F58
:102E000080831092E2001092DA001092E100A0EEAE
:102E1000B0E08C9181608C9380818F77808319BC26
:102E2000A7EDB0E08C918E7F8C9380818F7E808324
:102E30001092D3020895A0E0B0E0E1E2F7E10C9433
:102E40006F2BC8EDD0E088818F7E8883E7EDF0E0BE
:102E500080818160808384E082BF81E08093D3029F
:102E600088818E7F888302EE10E0F8011082109234
:102E7000DA0081EEC82ED12CF601108288818F777E
:102E8000888388818068888388818F7D888319BC46
:102E90001092E0021092E1021092DF021092DE0224
:102EA00090EEE92EF12CF70180818B7F8083888161
:102EB0008160888342E060E080E00E94E412F601D5
:102EC00080818E7F8083F801808181608083808112
:102ED00088608083F70180818E7F80838881806114
:102EE0008883CDB7DEB7E8E00C948B2B1F920F924E
:102EF0000FB60F9211242F933F934F935F936F93CD
:102F00007F938F939F93AF93BF93EF93FF938091A2
:102F1000E10082FF49C08091E20082FF45C08091BC
:102F2000E1008B7F8093E1002091D2022F5F822FFE
:102F300062E30E94382B992319F02093D20234C007
:102F40001092D2028091D102882371F18091E00227
:102F5000843041F58091E9008F702091EC00922F30
:102F6000917020FD90E8892B95E09093E900909175
:102F7000EB0090FF14C09091EE0097FF10C090916D
:102F8000E80095FF03C01092F100F9CF9091E8009E
:102F900090FF05C09091E8009E779093E8008F70B5
:102FA0008093E9001092D1028091DA0080FF3AC04C
:102FB0008091D80080FF36C08091DA008E7F8093A8
:102FC000DA008091D90080FF20C080E189BD82E1D4
:102FD00089BD09B400FEFDCF81E08093E0028FE15E
:102FE00094E09F938F930E9402088091D3020F90E8
:102FF0000F90811117C00E94FC160E941B17809130
:10300000E20084608093E2000DC019BC1092E002DF
:1030100083E294E09F938F930E9402081092D30260
:103020000F900F908091E10080FF1FC08091E2001F
:1030300080FF1BC08091E2008E7F8093E200809130
:10304000E20080618093E2008091D80080628093EA
:10305000D80019BC85E08093E00287E294E09F935A
:103060008F930E9402080F900F908091E10084FFDF
:1030700038C08091E20084FF34C080E189BD82E1E4
:1030800089BD09B400FEFDCF8091D8008F7D80936B
:10309000D8008091E1008F7E8093E1008091E20072
:1030A0008F7E8093E2008091E20081608093E20055
:1030B0008091E102882311F084E007C08091E30051
:1030C00087FD02C081E001C083E08093E0028BE2D3
:1030D00094E09F938F930E9402088091E0020F90EA
:1030E0000F908091E10083FF2FC08091E20083FF69
:1030F0002BC08091E100877F8093E10082E0809384
:10310000E0021092E1028091E1008E7F8093E10065
:103110008091E2008E7F8093E2008091E2008061E6
:103120008093E20042E060E080E00E94E41280913F
:10313000F00088608093F0008FE294E09F938F937B
:103140000E9402080F900F90FF91EF91BF91AF91F5
:103150009F918F917F916F915F914F913F912F91AF
:103160000F900FBE0F901F9018952091E4003091A2
:10317000E50095E64091EC00842F817040FF23C06C
:103180008091E80080FD1DC08091E002882399F0C5
:10319000853099F08091EB0085FD11C04091E400ED
:1031A0005091E5002417350729F3915011F09A0149
:1031B000E1CF84E0089582E0089583E0089581E0FE
:1031C000089580E008954091E80042FFDDCF089522
:1031D0002091480390910F0357E02917A9F030E0A0
:1031E000529FF001539FF00D1124E05FFC4F71815D
:1031F000761306C07081781303C07581741306C0FE
:103200002F5F3F4F2770E9CF80E0089581E0089558
:103210009091740380914B03892B90914A039923D9
:10322000E1F0892B90910A01992341F09091BA0322
:1032300097FF04C09EE125E833E003C096E02DE748
:1032400033E0F90120E0915028F031913323D9F394
:103250002F5FF9CF211110924A03089580914803FE
:1032600090910F03891719F08F5F8770FBCF089536
:10327000CF93DF9380910E0382958F7009F04EC03B
:1032800080910D03882309F449C08091480340913F
:103290000F035091090360910803C0910A03D09174
:1032A0000B0377E08417D1F190E0789FF001799FCC
:1032B000F00D1124DF01A05FBC4F14962C911497E0
:1032C000222349F111962C911197251324C02C919A
:1032D000261321C015962C91159721111CC012960A
:1032E0002D913C9113972C1B3D0B283C310598F4F4
:1032F00080910E038F70806180930E03EA5EFC4F15
:1033000080818F708061808388E093E00E94E8086C
:103310000E942E1903C001968770C4CFDF91CF9110
:103320000895CF92DF92FF920F931F93CF93DF9375
:103330006C010091BA0280917503082BC3E0D0E0C4
:1033400010E0C8010C2E02C0959587950A94E2F70B
:1033500080FD04C02197A8F7F12C09C0FC2EB6010E
:103360008C2F0E94D91F0E94E71F019799F38F2D80
:10337000DF91CF911F910F91FF90DF90CF90089533
:10338000CF93DF93EC010E949119BE010E94D91FD7
:103390000E94E71FDF91CF910895FC012481222331
:1033A000D9F0808191810E94C01992959F709630CA
:1033B00079F010F4925001C09A50923068F4803F36
:1033C00069F018F4883E40F409C0843F29F406C02F
:1033D000883E20F0813F11F080E0089581E008955B
:1033E000A4E1B0E0E6EFF9E10C946B2B8C0186E0F0
:1033F000F801DE011F9601900D928A95E1F7F80120
:103400008481E58098E0892E93E0992E90910C03B9
:10341000911120C0882309F463C1EE2009F442C051
:10342000C8010E94CD19F82E8823E1F187E0F80148
:10343000D40101900D928A95E1F780910C038130BF
:1034400031F480910803909109030E94C0190E94F1
:10345000381948C1F801D080C180A280B380F090B3
:103460000D0320910A0330910B03FF2009F4E7C0FC
:10347000A501421B530B483C510508F09DC0882311
:1034800009F430C180910E03282F207F9091090309
:10349000222361F09C1509F460C0C8010E94CD1977
:1034A000811163C0C8010E94E8081AC19C1113C0B1
:1034B000909108039D110FC0E1100DC08F708061C5
:1034C00080930E0388E093E00E94E80880910E0349
:1034D000F801868303C1E1103AC040E06C2D8D2DC8
:1034E0000E94E81840E06C2D8D2D0E94E818E82E0F
:1034F0008111F4C0DF86C88A8F8598890E94C0191F
:10350000292F22952F70243020F49F70223028F02C
:1035100009C02A50223080F014C0992349F081114B
:1035200007C013C0992321F0F8019681907F69F0BC
:10353000805E883030F409C0803F38F0815F83308E
:1035400020F0C8010E94E808EF2CFE2CCBC080912F
:103550000E03816080930E03C1C0909108039D11FA
:103560009CCFE1109ACFF80198C0EE2009F49ACFD1
:1035700020910E03822F82958F7090E002978CF03D
:10358000809108039091090399878887BB86AA8652
:1035900080910C038C871D862E87CE0108960E9491
:1035A000E80887E0F801A8E0B3E001900D928A9561
:1035B000E1F70E94381994C090910E03292F207FC3
:1035C00051F488E093E00E94E80887E0F40111924A
:1035D0008A95E9F783C0882309F484C080910903A0
:1035E0008C110CC0809108038D1108C0E11006C039
:1035F000F8019683C8010E94E8086AC0C8010E94C9
:10360000CD19882309F44ECFEE2009F44BCF209139
:103610000E03822F82958F7090E0029714F28091B2
:103620000803909109039A838983BC82AB828091BD
:103630000C038D831E822F83CE010196B0CFA21A78
:10364000B30AF8ECAF16B10408F042C0882309F4BD
:1036500047C0FE2CEE2009F425CF809109038C1180
:1036600029C0809108038D1125C090910E0390FD13
:1036700018C0892F82958F70282F30E021153105D1
:1036800081F0F80196832F30310541F08F5F982F3C
:103690009295907F86818F70892B8683C8010E94C6
:1036A000E80887E0F801A8E0B3E001900D928A9560
:1036B000E1F718C0C8010E94CD19811172CF809125
:1036C0000E03816080930E03C8010E94E8080AC0BF
:1036D00087E0F40111928A95E9F704C0F12C02C049
:1036E000FF24F3948F2D6496ECE00C94872B292F04
:1036F000953078F58F3068F590E03FE0239F800D9E
:10370000911D1124682F677023E0969587952A955F
:10371000E1F7FC01EE0FFF1FE80FF91FE651FD4F27
:1037200040E050E080E0219130E0062E02C0369566
:1037300027950A94E2F721703327042E01C0220F47
:103740000A94EAF7822B4F5F5F4F4330510559F7D8
:10375000089580E00895292F953088F58F3078F509
:1037600090E03FE0239F800D911D1124282F2770AA
:1037700051E001C0550F2A95EAF723E09695879509
:103780002A95E1F7FC01EE0FFF1FE80FF91FE65144
:10379000FD4F20E030E070E04081CB01022E02C0FE
:1037A000969587950A94E2F7817081958427852301
:1037B000842781932F5F3F4F2330310569F70895A8
:1037C0008093BA0208959091BA0221E030E0F901A5
:1037D00001C0EE0F8A95EAF7D90102C0AA0FBB1FFC
:1037E0006A95E2F7BD016E2B01C0220F4A95EAF7F8
:1037F000892F8623681303C0892F822B03C020954D
:10380000822F89230E94E01B089521E030E001C04F
:10381000220F8A95EAF720958091BA0282230E94AE
:10382000E01B089590914903809589238093490373
:10383000282F277069F4981759F09091BB0392FFD5
:1038400007C08695869586950E94051C10924903AF
:103850000895CF939091BB0392FB222720F928175C
:1038600009F1C82F892FC0FB82F98093BB036091B7
:10387000BA037091BB0384E090E00E94222B82E0A7
:103880000E94121C8091B90380FF0CC01F92CF933D
:103890008FEF94E09F938F930E9402080F900F90F8
:1038A0000F900F90CF91089521E030E001C0220FDA
:1038B0008A95EAF78091BA02822B0E94E01B089554
:1038C0008093750308951092740380910A018823F0
:1038D00041F08091BA0387FF04C08EE1E5E8F3E090
:1038E00003C086E0EDE7F3E0DF011D928A95E9F77A
:1038F00080E090E00E94122480E090E00E94ED239E
:1039000010924B030E949C21EAEAF3E086E0DF017B
:103910001D928A95E9F71092A5031092A3031092C5
:10392000A4030E9405250895882321F00E94952173
:103930000E949C210895882339F090917403892B6B
:10394000809374030E949C210895882309F456C033
:10395000823859F40E94372481FF50C089E30E94C5
:10396000A5230E949C2189E30CC0833879F40E942E
:10397000372480FF43C083E50E94A5230E949C2139
:1039800083E50E9466230E949C210895843859F49F
:103990000E94372482FF32C087E40E94A5230E9440
:1039A0009C2187E4EECF9CEF980F913A50F390E280
:1039B000980F983050F4877091E001C0990F8A9564
:1039C000EAF7892F0E949521DECF9BE5980F93306F
:1039D00028F480E090E00E941224089598E5980F62
:1039E0009B3128F480E090E00E94ED23089593E35A
:1039F000980F933118F460E00E94FA290895CF934C
:103A0000882309F407C1C82F8238A1F40E94372403
:103A100081FD00C189E30E94A5230E949C212FEF14
:103A200087EE93E0215080409040E1F700C0000015
:103A300089E315C08338C1F40E94372480FDEAC0B1
:103A400083E50E94A5230E949C212FEF81EE94E044
:103A5000215080409040E1F700C0000083E50E94C3
:103A600066230E949C21D6C08438A1F40E9437248A
:103A700082FDD0C087E40E94A5230E949C212FEFE5
:103A800081EE94E0215080409040E1F700C00000BA
:103A900087E4E5CF8CEF8C0F813A08F04BC0809122
:103AA000C103813089F038F0823009F040C08C2F9A
:103AB0000E943927AFC080917403823209F076C02A
:103AC0008C2F0E946C2870C0809174038232C1F3E5
:103AD000C43109F158F4CB3069F0C031F9F482E017
:103AE0008093C10388E30E94392759C0C93299F0F5
:103AF000C833A1F48FE49BE09F938F930E94020848
:103B00008BEF94E09F938F930E9402080F900F9089
:103B10000F900F9044C01092C10344C089EF94E00D
:103B20009F938F930E9402080F900F903BC01092BA
:103B3000C1033CC080E28C0F883068F4C77081E01C
:103B400090E001C0880FCA95EAF790917403892B21
:103B50008093740386CFEBE5EC0FE33040F4F0E0A4
:103B6000E75CFE4F808190E00E94122453C0E8E59C
:103B7000EC0FEB3150F4F0E0EE0FFF1FE45CFE4F72
:103B8000808191810E94ED2345C083E38C0F8331B6
:103B900008F040C061E08C2F0E94FA293BC081E010
:103BA000817002C080E0FCCF811134C080910A0195
:103BB0008823E1F08091BA0387FF18C0EC2FE695C7
:103BC000E695E695F0E0ED57FC4F8281282F30E036
:103BD0004C2F477081E090E002C0880F991F4A95F2
:103BE000E2F782239323892B61F410C0EDE7F3E021
:103BF00083E893E02191C21721F08E179F07D1F738
:103C000005C08C2F0E9466230E949C218C2F0E944D
:103C1000A52327CFCF9108951F93CF93DF93182F1C
:103C2000EB010E94FF1C209741F08FE99FE0019774
:103C3000F1F700C000002197F6CF812F0E94A51C4C
:103C4000DF91CF911F9108959091BA0392FF10C018
:103C500041E0282F2471243009F040E031E0282F82
:103C60002871283009F030E0431711F02CE082274A
:103C700093FF10C041E0282F2471243109F040E067
:103C800031E0282F2871283109F030E0431711F076
:103C90002CE082273091BB0330FF10C051E0282F69
:103CA0002171213009F050E041E0282F287128309F
:103CB00009F040E0541711F029E0822731FF10C0CD
:103CC00041E0282F2171213109F040E031E0282F17
:103CD0002871283109F030E0431711F029E08227DC
:103CE00094FD877E08958238910569F1B0F481339F
:103CF000910509F475C048F48932910509F467C04B
:103D00008A32910509F471C008958533910509F44B
:103D100059C089339105B9F00895833E910589F121
:103D200038F4803E9105D1F0823E910529F1089545
:103D3000863E9105C9F1873E9105D9F1843E9105F2
:103D400009F06CC027C02091BA0320FD57C021FDA7
:103D500055C02091BB0323FD5BC008958091BA0339
:103D600080FD48C08091BB0380FF48C08091BA03AA
:103D700084FD46C083EE51C08091BA0382FF3CC0EF
:103D8000F5CF8091BA0382FD37C08091BB0380FDDF
:103D900035C0ECCF8091BB0381FF36C08091BA0360
:103DA00084FD2EC087EE39C08091BA0383FF2AC0FC
:103DB000F5CF8091BA0383FD25C08091BB0381FDBF
:103DC00023C0ECCF8091BA0385FD22C01FC0809133
:103DD000BA0385FD1BC08091BB0383FF19C00AC0D5
:103DE0008091BA0386FD16C017C08091BA0386FD84
:103DF00013C010C089E311C082EE0FC080EE0DC069
:103E000080E00BC086EE09C084EE07C085E305C0E4
:103E100089E203C08AE201C081E390E00895F8944A
:103E2000E82FE295EF70F0E031A1282F2F7081E0AC
:103E300090E001C0880F2A95EAF7982F9095932378
:103E400091A392A1892B82A378940895AAE0B0E06F
:103E5000ECE2FFE10C94692BAE014F5F5F4F7A01FA
:103E60008AE0FA0111928A95E9F701E111E06A010D
:103E700096E1692E91E0792E88248394912CF801A3
